:020000040800F2
:10000000D005002031020008151F0008B71E0008A7
:10001000111F00086D070008692400080000000097
:10002000000000000000000000000000FF1F0008AA
:10003000D909000800000000FD1F00080120000889
:100040005502000855020008550200085502000834
:100050005502000855020008550200085502000824
:100060005502000855020008550200085502000814
:100070005502000855020008550200085502000804
:1000800055020008550200085502000855020008F4
:1000900055020008550200085502000855020008E4
:1000A00055020008550200085502000855020008D4
:1000B00055020008550200085502000855020008C4
:1000C00055020008550200085502000855020008B4
:1000D00055020008192400085502000855020008BE
:1000E0005502000855020008550200085502000894
:1000F0005502000855020008550200085502000884
:100100005502000855020008550200085502000873
:100110005502000855020008550200085502000863
:100120005502000855020008550200085502000853
:100130005502000855020008550200085502000843
:100140005502000855020008550200085502000833
:100150005502000855020008550200085502000823
:100160005502000855020008550200085502000813
:100170005502000855020008550200080000000062
:10018000550200085502000800F002F800F041F89E
:100190000AA090E8000C82448344AAF10107DA45E2
:1001A00001D100F036F8AFF2090EBAE80F0013F0F3
:1001B000010F18BFFB1A43F001031847282900005C
:1001C00048290000103A24BF78C878C1FAD85207ED
:1001D00024BF30C830C144BF04680C6070470000C1
:1001E0000023002400250026103A28BF78C1FBD840
:1001F000520728BF30C148BF0B607047782900F014
:10020000F580002070471FB502F046FC1FBD10B5F9
:1002100010BD00F0C9F91146FFF7F5FF02F0D8F95B
:1002200000F0E7F903B4FFF7F2FF03BC02F03AF97C
:100230000C48016841F4700101600B4880470B488D
:100240000047FEE7FEE7FEE7FEE7FEE7FEE7FEE724
:10025000FEE7FEE7FEE7000005480649044A064BB4
:100260007047000088ED00E00920000889010008BF
:10027000D0010020D0050020D0010020704753EAB3
:10028000020C00F069802DE9F04B4FF00006002BC6
:100290001FBFB3FA83F503FA05F424FA05F65E40AE
:1002A00012BF1643B2FA82F502FA05F4C5F1200531
:1002B0001EBF22FA05FC44EA0C04203556EA044C21
:1002C0004FEA144418BF641C4FF000084FF00009B7
:1002D000904271EB030C39D3002919BFB1FA81F7B1
:1002E00001FA07F6B0FA80F700FA07F6C7F120071F
:1002F0001EBF20FA07FC46EA0C062037B6FBF4FCCA
:10030000A7EB0507103F07F01F0BCBF120060CFAF7
:100310000BFB2CFA06F644BFB3460026202FA4BFE1
:100320005E464FF0000B5BEA060C08BF4FF0010B76
:1003300019EB0B09ABFB027C48EB0608C01B06FB64
:1003400002CC0BFB03CC71EB0C01C1E70B46024660
:1003500041464846BDE8F08B13B54FF000004FF022
:100360000001AFF30080BDE81C4070470FB40449A2
:1003700010B503AA029800F0E9F810BC5DF814FB70
:10038000080000202DE9F0410E46044600202062BE
:100390002046E168884730B3252805D0D4E90121FB
:1003A0009047206A401CF2E7E16820460027884712
:1003B000050018D0A5F14100192802D820354FF4C6
:1003C00000673246294620462760FFF717FF40B1F5
:1003D000012804D0F61D26F007060836D8E7361D9A
:1003E000D6E72846DAE7206ABDE8F08170B5044612
:1003F0000D4621461068AFF300802188090502D51B
:100400000F4A7A4402E00E4A7A440E32002104F187
:10041000240305E000F00F060009965D5E54491CB8
:100420000028F7D120780023000704D5702D02D0D2
:1004300009B1022311322046BDE8704000F02DB80A
:10044000B42600004FF0000200B5134694469646CD
:10045000203922BFA0E80C50A0E80C50B1F12001D7
:10046000BFF4F7AF090728BFA0E80C5048BF0CC085
:100470005DF804EB890028BF40F8042B08BF7047E3
:1004800048BF20F8022B11F0804F18BF00F8012B55
:10049000704770477047704770472DE9F0470D4629
:1004A00099469246044600F124080168880604D55E
:1004B000E06921F01001216000E00120A84201DD87
:1004C000471B00E00027A1697A1902EB0900081A0E
:1004D000A0612078C00602D42046AFF30080002639
:1004E00008E0D4E901211AF806009047206A401C70
:1004F000761C20624E45F4DB2078C0060AD52046E3
:10050000AFF3008006E0D4E9012130209047206A53
:10051000401C2062381EA7F10107F4DC07E0D4E993
:10052000012118F805009047206A401C2062281E0F
:10053000A5F10105F3DC2046AFF30080207800062A
:1005400002D50220BDE8F0870120FBE7074B70B51C
:100550000D467B4400F011F80446284600F020F8D0
:1005600010B14FF0FF3070BD204670BD5F2000001D
:1005700001694A1C02610878704700B58FB0CDE967
:1005800001310021059105497944CDE90310114657
:100590006846FFF7F7FE0FB000BD0000E5FFFFFF64
:1005A000007B00F080007047754600F02BF8AE46E7
:1005B00005006946534620F00700854618B020B56F
:1005C000FFF74AFEBDE820404FF000064FF000075D
:1005D0004FF000084FF0000B21F00701AC46ACE8EB
:1005E000C009ACE8C009ACE8C009ACE8C0098D4658
:1005F000704710B50446AFF300802046BDE81040B8
:10060000FFF710BE004870477001002055494A6846
:1006100022F440324A604A6843681A434A600268DA
:10062000526822F4807203685A6002685368026953
:1006300043EA022203685A600268526822F040725C
:1006400003685A600268526883681A4303685A60F4
:100650000268926822F4006203689A6002689268F5
:10066000C3681A4303689A603F4B826A9A4218D063
:100670000268926822F0706203689A600268926869
:10068000836A1A4303689A600268926822F04052B3
:1006900003689A6002689268C36A1A4303689A60A2
:1006A0000BE00268926822F0706203689A60026848
:1006B000926822F0405203689A600268926822F0C1
:1006C000020203689A6002689368027E43EA42026B
:1006D00003689A602022125CA2B10268526842F458
:1006E000006203685A600268526822F4604203683C
:1006F0005A6002685368426A521E43EA42320368F3
:100700005A6005E00268526822F4006203685A6089
:100710000268D26A22F470020368DA620268D36A5D
:10072000828B521E43EA02520368DA6202689268C0
:1007300022F4007203689A600268936890F830208F
:1007400043EA422203689A600268926822F4806257
:1007500003689A6002689368426943EA82220368E8
:100760009A607047002301400100000F00BFFEE7C0
:1007700000B587B0142102A8FFF764FE00BF002077
:1007800001903848006840F010003649086008467B
:10079000006800F01000019000BF00BF00BF002003
:1007A00001900846006840F00400086008460068B0
:1007B00000F00400019000BF00BF00BF00200190C6
:1007C0000846006840F0200008600846006800F015
:1007D0002000019000BF00BF00221C21224800F031
:1007E000B5FC01226021204800F0B0FC00224FF44B
:1007F00000511E4800F0AAFC002222211C4800F0F3
:10080000A5FC1C200290012003900020049005907C
:1008100002A9154800F098FB602002900120039087
:10082000002004900120059002A90F4800F08CFBE5
:100830004FF4005002900120039000200490059096
:1008400002A90A4800F080FB2220029001200390B8
:1008500000200490059002A9054800F075FB07B040
:1008600000BD000030380240001002400008024085
:100870000014024070B505460C46012D3DD1002103
:1008800000F098F800221C21474800F05FFC092C7A
:1008900031D2DFE804F03005060C12181E242A00BD
:1008A0002AE001220421404800F050FC24E001220B
:1008B00008213D4800F04AFC1EE001220C213A4884
:1008C00000F044FC18E001221021374800F03EFC03
:1008D00012E001221421344800F038FC0CE001221F
:1008E0001821314800F032FC06E001221C212E487C
:1008F00000F02CFC00E000BF00BF022D52D101210E
:10090000002000F057F800222903284800F01EFCC0
:1009100000222221264800F019FC092C40D2DFE8F1
:1009200004F03F05060C121D232E340039E001228D
:1009300051031E4800F00AFC33E0012202211C484A
:1009400000F004FC2DE001220221194800F0FEFB1A
:1009500001225103154800F0F9FB22E00122202179
:10096000134800F0F3FB1CE0012251030F4800F094
:10097000EDFB012220210E4800F0E8FB11E00122EE
:1009800022210B4800F0E2FB0BE001225103074853
:1009900000F0DCFB01222221054800F0D7FB00E03B
:1009A00000BF00BF70BD0000001002400008024000
:1009B0000014024070B504460D4684F00102202167
:1009C000044800F0C3FB85F001024021014800F01B
:1009D000BDFB70BD001002407047000038B50246F4
:1009E0000020009000BF92F83C00012801D10220B5
:1009F00038BD012082F83C0000BF0868092816D9DC
:100A00001068C0680C780A3C04EB44050724AC402D
:100A1000A0431468E0600C780A3C04EB4404886846
:100A2000A0401468E46820431468E06013E0106894
:100A300000690C7804EB44050724AC40A04314681B
:100A400020610C7804EB44048868A0401468246991
:100A50002043146820614868072817D21068406B4B
:100A60000C79641E04EB84051F24AC40A043146879
:100A70006063088880B20C79641E04EB8404A04093
:100A80001468646B20431468606331E048680D2883
:100A900017D21068006B0C79E41F04EB84051F2447
:100AA000AC40A04314682063088880B20C79E41F2E
:100AB00004EB8404A0401468246B20431468206372
:100AC00016E01068C06A0C790D3C04EB84051F2405
:100AD000AC40A0431468E062088880B20C790D3CF9
:100AE00004EB8404A0401468E46A20431468E062C4
:100AF000194B1A4C1068A04206D10868122803D17D
:100B0000586840F480005860144C1068A0421CD112
:100B10000868102802D00868112816D1586840F4D7
:100B200000005860086810280FD10D4800680D4C6F
:100B3000B0FBF4F000EB80004000009002E0009871
:100B4000401E009000980028F9D100BF002082F8D4
:100B50003C0000BF00BF4BE70023014000200140E4
:100B60000000002040420F0001460868C06C70473A
:100B700070B5044600250CB9012070BD1549A06A66
:100B8000884200D000BF206C30B9204600F024F825
:100B90000020606484F83C00206C00F0100088B9EC
:100BA000206C20F4885040F0020020642046FFF7BB
:100BB0002DFD00206064206C20F0020040F0010058
:100BC000206400E0012500BF002084F83C0000BF45
:100BD0002846D2E70100000F10B586B00446142164
:100BE00001A8FFF72FFC1949206888422BD100BFCC
:100BF000002000901648006840F4806014490860A6
:100C00000846006800F48060009000BF00BF00BF8D
:100C1000002000900E481438006840F020000C4975
:100C2000143908600846006800F02000009000BFFA
:100C300000BF18200190032002900020039001A91A
:100C4000044800F081F906B010BD00000022014008
:100C5000443802400014024070B504460D46002698
:100C60002068806800F48060B0F5806F11D1206842
:100C7000806800F48070B0F5807F0AD1206C40F06D
:100C80002000206400BF002084F83C0000BF012049
:100C900070BD00F067FA064618E0681CB0B125B1D7
:100CA00000F060FA801BA84210D92068006800F0AC
:100CB000020002280AD0206C40F00400206400BF2B
:100CC000002084F83C0000BF0320E1E720680068B2
:100CD00000F002000228E0D16FF0120021680860E5
:100CE000206C40F4007020642068806800F0405060
:100CF000B8B9207EA8B92068C06A00F4700020B19D
:100D00002068806800F4806058B9206C20F48070FE
:100D10002064206C00F4805018B9206C40F0010071
:100D200020640020B4E7000008B5014600200090D0
:100D300000BF91F83C00012801D1022008BD01202C
:100D400081F83C0000BF0868806800F00100A0B98D
:100D50000868806840F001000B6898603F480068B0
:100D60003F4BB0FBF3F000EB4000009002E0009836
:100D7000401E009000980028F9D10868806800F0B3
:100D80000100002860D0086C40F20163984340F4F1
:100D9000807008640868406800F4806028B1086CBE
:100DA00020F4005040F480500864086C00F4805037
:100DB000B0F5805F04D1486C20F00600486401E083
:100DC0000020486400BF002081F83C0000BF254A95
:100DD0006FF022000B681860506800F01F0018BB0D
:100DE000214B0868984213D0204B0868984204D1E0
:100DF000101D006800F01F0050B11D4B086898429C
:100E00002AD11848001D006800F01F00102823D2C6
:100E10000868806800F04050F0B90868806840F0C9
:100E200080400B68986017E00F4B0868984213D118
:100E30000868806800F0405070B90868806840F029
:100E400080400B68986007E0086C40F01000086470
:100E5000486C40F00100486400206FE7000000206B
:100E600040420F00002301400020014000210140CA
:100E70000022014070B50446A56D00F073F90646E6
:100E800094F83500022808D08020606500BF00205B
:100E900084F8340000BF012070BD2068006820F095
:100EA0001600216808602068406920F080002168F1
:100EB0004861206C08B9A06C28B12068006820F057
:100EC0000800216808602068006820F0010021689F
:100ED00008600FE000F046F9801B05280AD92020A1
:100EE000606500BF002084F8340000BF032084F850
:100EF0003500D1E72068006800F001000028E9D142
:100F000094F85C103F208840A86000BF002084F85F
:100F1000340000BF012084F835000020BCE7014602
:100F200091F83500022803D08020486501207047E1
:100F3000052081F835000868006820F001000A6883
:100F400010600020F3E70000F8B502460B460025CC
:100F5000002400200021DEE0012606FA01F51E68CB
:100F600006EA0504AC4275D11E7906F00306012E8F
:100F700004D01E7906F00306022E13D190684F00AC
:100F80000326BE40B0434F00DE68BE403043906051
:100F9000506801268E40B0431E79C6F300168E407D
:100FA000304350601E7906F00306032E09D0D06846
:100FB0004F000326BE40B0434F009E68BE40304302
:100FC000D0601E7906F00306022E13D1CF0802F17D
:100FD000200656F827004E07F70E0F26BE40B043F6
:100FE0004F07FF0E1E69BE403043CF0802F12006B6
:100FF00046F8270010684F000326BE40B0431E7914
:1010000006F003064F00BE40304310605E6806F0F5
:101010008056B6F1805F7DD100BF00260096404E1D
:10102000366846F480463E4F3E603E46366806F4DB
:101030008046009600BF00BF3A4E8F0856F8270042
:101040008E07370F0F26BE40B043374EB24202D153
:10105000002624E05EE0354EB24201D101261EE0BA
:10106000334EB24201D1022619E0324EB24201D1D2
:10107000032614E0304EB24201D104260FE02F4E79
:10108000B24201D105260AE02D4EB24201D1062618
:1010900005E02C4EB24201D1072600E008268F075A
:1010A0003F0FBE4030431F4E8F0846F82700264EA4
:1010B0003068A0435E6806F48036B6F5803F00D104
:1010C0002043214E3060361D3068A0435E6806F430
:1010D0000036B6F5003F00D120431B4E361D306070
:1010E000361D3068A0435E6806F48016B6F5801F92
:1010F00000D12043144E08363060361D3068A043BE
:101100005E6806F40016B6F5001F00D120430E4EAF
:101110000C363060491C1029FFF41EAFF8BD0000EA
:1011200044380240083801400000024000040240F8
:1011300000080240000C024000100240001402406F
:1011400000180240001C0240003C01400AB18161CD
:1011500001E00B048361704701480068000C704790
:10116000002004E0014800687047000010000020E3
:10117000034800680349097808440149086070473A
:10118000100000201800002010B50A48006840F444
:101190000070084908600846006840F480600860F4
:1011A000032000F07FF80F2000F006F800F02AF886
:1011B000002010BD003C024070B504460E48007887
:1011C0004FF47A71B1FBF0F00C490968B1FBF0F50E
:1011D000284600F01DFC08B1012070BD102C07D27C
:1011E00000222146501E00F01EF80548046001E070
:1011F0000120F2E70020F0E71800002000000020A6
:1012000014000020704701460846002809DB00F062
:101210001F0301229A4043099B0003F1E023C3F816
:10122000002100BF70472DE9F05F80460D4616464D
:10123000002701F01BF9074639462A46334601F0DC
:101240000700C0F1070ABAF1040F02D94FF0040AEF
:1012500001E0C0F1070AD14600F1040ABAF1070F14
:1012600002D24FF0000A01E0A0F1030AD4464FF089
:10127000010A0AFA09FAAAF1010A0AEA020A0AFAB2
:101280000CFA4FF0010B0BFA0CFBABF1010B0BEA64
:10129000030B4AEA0B042146404601F0EFF8BDE893
:1012A000F09F000000BF00F00702064B19684FF6E0
:1012B000FF031940044B0B4343EA0221014B196021
:1012C00000BF70470CED00E00000FA0570B5044661
:1012D0000D460CB9012070BD5848006800F00700A9
:1012E000A84209D255490D700846006800F0070071
:1012F000A84201D00120EEE7207800F00200022889
:101300001DD1207800F00400042805D14C48006865
:1013100040F4E0504A490860207800F008000828AE
:1013200005D14748006840F460404549086044489A
:10133000006820F0F000A168084341490860207867
:1013400000F00100A8B36068012807D13C480838C4
:101350000068C0F34040B8B90120BCE760680228CB
:1013600002D06068032807D1354808380068C0F308
:10137000406048B90120AEE7314808380068C0F342
:10138000400008B90120A6E72D48006820F00300BE
:10139000616808432A490860FFF7E4FE064609E051
:1013A000FFF7E0FE801B41F28831884202D903201A
:1013B00091E707E02248006800F00C006168B0EB9C
:1013C000810FEDD11D48006800F00700A84209D93F
:1013D0001A490D700846006800F00700A84201D0C5
:1013E000012078E7207800F00400042807D1144891
:1013F000006820F4E050E168084311490860207853
:1014000000F00800082808D10D48006820F460406A
:10141000216940EAC1000A49086000F03FF8084924
:101420000968C1F30311074A515CC84006490860C6
:1014300006480068FFF7C0FE00204CE7003C024071
:1014400008380240A22A00080000002014000020F2
:1014500001480068704700000000002000B5FFF759
:10146000F7FF04490968C1F38221034A515CC8406F
:1014700000BD000008380240B22A000800B5FFF79E
:10148000E7FF04490968C1F34231034A515CC8408F
:1014900000BD000008380240B22A00082DE9F047DC
:1014A000002400250026A1462548006800F00C0015
:1014B00020B1042805D008283AD105E0DFF884904F
:1014C00039E0DFF8849036E01D48001F006800F026
:1014D0003F041B48001F006800F4800078B11A48E0
:1014E0001749091F0968C1F38811A0FB0170014663
:1014F000224600233846FEF7C2FE05460EE011489C
:101500000F49091F0968C1F38811A0FB017001464A
:10151000224600233846FEF7B2FE05460848001F63
:101520000068C0F30140401C4600B5FBF6F902E03C
:10153000DFF8109000BF00BF4846BDE8F08700000C
:10154000083802400024F40000127A00F8B504467E
:101550000CB90120F8BD207800F00100002874D0FB
:10156000F948006800F00C0004280DD0F648006827
:1015700000F00C00082813D1F348001F006800F4A5
:101580008000B0F5800F0BD1EF4808380068C0F339
:101590004040002859D06068002856D10120D9E782
:1015A00000BF6068B0F5803F08D1E74808380068A0
:1015B00040F48030E449083908601EE06068B0F506
:1015C000A02F0DD1E0480838006840F48020DE49A3
:1015D000083908600846006840F4803008600CE074
:1015E000D9480838006820F48030D74908390860A5
:1015F0000846006820F48020086000BF606890B151
:10160000FFF7B0FD054606E0FFF7ACFD401B642880
:1016100001D903209EE7CC4808380068C0F3404059
:101620000028F1D011E0FFF79DFD054606E0FFF729
:1016300099FD401B642801D903208BE7C248083874
:101640000068C0F340400028F1D1207800F002008B
:1016500002285FD1BC48006800F00C0058B1BA48BD
:10166000006800F00C0008281CD1B748001F006873
:1016700000F48000B0B9B44808380068C0F34000F6
:1016800020B1E068012801D0012063E7AE480838A6
:10169000006820F0F800216940EAC100AA49083931
:1016A000086037E0E06800B30120A8490860FFF750
:1016B00059FD054606E0FFF755FD401B022801D9FC
:1016C000032047E7A04808380068C0F3400000281E
:1016D000F1D09D480838006820F0F800216940EA00
:1016E000C10099490839086014E000209749086052
:1016F000FFF738FD054606E0FFF734FD401B0228E2
:1017000001D9032026E7904808380068C0F340005C
:101710000028F1D1207800F0080008282CD1606959
:10172000A8B101208A490860FFF71CFD054606E0C4
:10173000FFF718FD401B022801D903200AE7824861
:101740006C300068C0F340000028F1D014E00020A5
:101750007F490860FFF706FD054606E0FFF702FD3A
:10176000401B022801D90320F4E677486C3000685A
:10177000C0F340000028F1D1207800F004000428D4
:1017800070D1002770483830006800F0805090B960
:1017900000BF002000906C483830006840F0805056
:1017A0006949383108600846006800F080500090B0
:1017B00000BF00BF01276748006800F48070B0B91F
:1017C0006448006840F4807062490860FFF7CAFC12
:1017D000054606E0FFF7C6FC401B022801D903209E
:1017E000B8E65C48006800F480700028F2D000BFC2
:1017F000A068012808D154486830006840F0010012
:101800005149683108601DE0A06805280DD14E4897
:101810006830006840F004004B49683108600846B1
:10182000006840F0010008600CE04748683000683C
:1018300020F001004449683108600846006820F043
:101840000400086000BFA068A8B1FFF78BFC054644
:1018500009E0FFF787FC401B41F28831884202D93A
:10186000032077E626E0384868300068C0F340007F
:101870000028EED013E0FFF775FC054608E0FFF7FF
:1018800071FC401B41F28831884201D9032061E696
:101890002D4868300068C0F340000028EFD1012FC8
:1018A00007D129483830006820F080502649383167
:1018B000086000BFA069002845D02348006800F0F8
:1018C0000C0008285DD0A069022845D100201F49DE
:1018D0000866FFF747FC054606E0FFF743FC401BA0
:1018E000022801D9032035E6174808380068C0F3FC
:1018F00040600028F1D1D4E907010843616A40EA59
:1019000081110122A06AC2EB500041EA00412C2063
:10191000005D41EA00600C49091F086001200B4985
:101920000866FFF71FFC054606E0FFF71BFC401B9F
:10193000022801D903200DE6034808380068C0F3E7
:1019400040600028F1D049E00838024000004742DA
:10195000800E474200700040002021490866FFF7D2
:1019600001FC054606E0FFF7FDFB401B022801D9FC
:101970000320EFE51B480068C0F340600028F2D167
:101980002CE0A069012800D1E4E51648001D066896
:10199000A069012820D006F48001E06981421BD1B2
:1019A00006F03F01206A814216D147F6C0703040F0
:1019B000616AB0EB811F0FD106F440310122A06AA9
:1019C000C2EB5000B1EB004F06D106F070612C2045
:1019D000005DB1EB006F01D00120BBE50020B9E54F
:1019E0000000474200380240042808D14FF0E021AF
:1019F000096941F004014FF0E022116107E04FF066
:101A0000E021096921F004014FF0E02211617047E3
:101A100070B504462546681EB0F1807F01D30120D1
:101A20000FE0681E4FF0E02148610F214FF0FF30BA
:101A300000F024FD00204FF0E021886107200861BC
:101A4000002070BD7047704701460022002391F8C6
:101A50003D2091F83E3042EA030070472DE9F84FEF
:101A60000446206805682068C668206847694FF00A
:101A70000009CA4605F00F09B9F1000F0AD105F0B7
:101A8000200038B106F0200020B1204600F0FBFA1B
:101A9000BDE8F88FB9F1000F72D007F0010018B956
:101AA00006F4907000286BD005F0010030B106F408
:101AB000807018B1206C40F00100206405F0040033
:101AC00030B107F0010018B1206C40F00200206432
:101AD00005F0020030B107F0010018B1206C40F0B1
:101AE0000400206405F0080048B106F0200010B999
:101AF00007F0010018B1206C40F008002064206C51
:101B000070B305F0200028B106F0200010B1204687
:101B100000F0B9FA20684069C0F3801A206C00F028
:101B2000080010B9BAF1000F23D0204600F080FA67
:101B30002068406900F04000402816D120684069C4
:101B400020F0400021684861A06B50B15648A16B5D
:101B50000865A06BFFF7E3F910B1A06B016D884732
:101B60000CE02046FFF76FFF08E02046FFF76BFF11
:101B700004E02046FFF767FF0020206488E7FFE7C6
:101B8000206B012879D105F01000002875D006F0EF
:101B90001000002871D000BF00200090206800686D
:101BA000009020684068009000BF00BF2068406936
:101BB00000F04000402839D1A06B006840681FFA4F
:101BC00080F8B8F1000F30D0A08D40452DDDA4F88D
:101BD0002E80A06BC069B0F5807F1FD02068C068E0
:101BE00020F480702168C8602068406920F00100FE
:101BF000216848612068406920F040002168486100
:101C0000202084F83E00002020632068C06820F077
:101C100010002168C860A06BFFF72CF9A08DE28D41
:101C2000801A81B22046FFF70DFF31E7A08DE18DCC
:101C3000401A1FFA80F8E08DE8B1B8F1000F1AD011
:101C40002068C06820F490702168C86020684069EE
:101C500020F0010021684861202084F83E00002027
:101C600020632068C06820F010002168C8604146E9
:101C70002046FFF7E7FE0BE7FFE705F0800030B1F5
:101C800006F0800018B1204600F095FB00E705F053
:101C9000400030B106F0400018B1204600F0E3F9F2
:101CA000F6E600BFF4E600001D20000810B504466B
:101CB0000CB9012010BDA06900B100E000BF94F88C
:101CC0003D0028B9002084F83C00204600F028F8A8
:101CD000242084F83D002068C06820F4005021686A
:101CE000C860204600F02EFA2068006920F4904079
:101CF000216808612068406920F02A002168486155
:101D00002068C06840F400502168C860002020644A
:101D1000202084F83D0084F83E000020CAE700003F
:101D200010B586B004462D492068884254D100BFC2
:101D300000BF002000902A48006840F010002849A9
:101D400008600846006800F01000009000BF00BF67
:101D500000BF00BF00BF0020009021481438006879
:101D600040F008001E49143908600846006800F079
:101D70000800009000BF00BF00BF00BF00BF0020F0
:101D800000900846006840F00200086008460068BD
:101D900000F00200009000BF00BF00BF4020019093
:101DA0000220029001200390022004900720059059
:101DB00001A90C48FFF7C8F8802001900720059082
:101DC00001A90848FFF7C0F82520FFF71CFA0322F5
:101DD00011462520FFF727FA06B010BD001001407C
:101DE000443802400004024070B504460D461646D1
:101DF00094F83E00202816D105B10EB9012070BD1F
:101E000000BF94F83C00012801D10220F7E701202F
:101E100084F83C0000BF002020633246294620465B
:101E200000F0A6FAEBE70220E9E700001D4A01688E
:101E3000914236D11C49098801F4004189BB1A49F5
:101E4000098801F4804171B1184909780A2903D041
:101E50000021154A118024E01349098841F400410A
:101E6000114A11801DE0114909780D2906D10E494A
:101E7000098841F480410C4A118012E00B4909782D
:101E8000094A1288C2F30D02094B99540649098880
:101E9000491C054A118011460988C72901DD002126
:101EA00011807047001001400C0000200E0000203F
:101EB0001C000020704700BFFEE700001FB5002097
:101EC00000900190029003900E480F4908604FF473
:101ED0008030486041020C48816000210161017638
:101EE00080F82010C162094981620021C16001218E
:101EF000C161002180F8301001214161FEF738FEF8
:101F00001FBD000000220140280100200100000F39
:101F100000BFFEE7704700002DE9F0412DED048B76
:101F200082B0002600270124012500BF50E00125D2
:101F30004BE029462046FEF79DFC642000F0FAFAAB
:101F4000012C1FD10A21092000F0D4FA8046404616
:101F500000F01AFC41EC190B9FED240B53EC102BF5
:101F600000F066FC41EC180B9FED220B53EC102B9C
:101F700000F05CFD05D2C5F1080101208840304326
:101F8000C6B200BF022C1FD10A210E2000F0B2FA07
:101F90008046404600F0F8FB41EC190B9FED130B17
:101FA00053EC102B00F044FC41EC180B9FED110B8F
:101FB00053EC102B00F03AFD05D2C5F108010120C9
:101FC00088403843C7B200BF6D1C092DB1DB641CCB
:101FD000032CACDB8DF804608DF80570BDF804109F
:101FE000084602B0BDEC048BBDE8F08100000000A3
:101FF0000000843F333333333333FB3F7047704744
:1020000010B5FFF7B5F810BD0348006840F4700044
:10201000014908607047000088ED00E070B5054692
:10202000AC6B0020E085E0842046FFF70CFD70BD1E
:102030000168C96821F490710268D160016849693A
:1020400021F0010102685161016B012905D101688C
:10205000C96821F010010268D160202180F83E108B
:1020600000210163704710B504462068C06820F065
:1020700040002168C860202084F83D002046FFF71A
:1020800019FF002010BD70B5044694F83E002228C8
:1020900056D1A068B0F5805F0CD1206950B90025F9
:1020A000A66A20684068C0F308003080A06A801CDF
:1020B000A06215E0A56A0026A068B0F5805F03D095
:1020C000A06828B9206918B920684068287004E021
:1020D0002068406800F07F002870A06A401CA06261
:1020E000E08D401E80B2E08540BB2068C06820F0D3
:1020F00020002168C8602068C06820F480702168D2
:10210000C8602068406920F00100216848612020F3
:1021100084F83E00206B01280AD12068C06820F0B6
:1021200010002168C860A18D2046FFF78BFC02E0FB
:102130002046FFF77BFE0020206370BD0020FCE7F7
:102140000220FAE72DE9F84F04462068006920F4E0
:102150004050E1680843216808612169A06808438C
:1021600061690843E169084300902068C06849F24A
:102170000C618843009908432168C8602068406961
:1021800020F44070A16908432168486176492068BD
:10219000884203D075492068884203D1FFF76EF961
:1021A000814602E0FFF75AF98146E069B0F5004F39
:1021B0006CD102206168A0FB015003461920A9FBE5
:1021C000007001462A463846FEF759F86421B0FBF4
:1021D000F1F04FEA001A02206168A0FB01510B46A2
:1021E0001920A9FB00712A463846FEF748F88346B5
:1021F00002206168A0FB015003461920A9FB007171
:102200002A463846FEF73BF86421B0FBF1F000EBBC
:10221000C00101EB0010ABEB8000322101EBC000EC
:102220006421B0FBF1F000F0F8000AEB400A022054
:102230006168A0FB015003461920A9FB007001460C
:102240002A463846FEF71BF8834602206168A0FB49
:10225000015003461920A9FB00712A463846FEF7B3
:102260000EF86421B0FBF1F000EBC00101EB0010AF
:10227000ABEB8000322101EBC0006421B0FBF1F038
:1022800000F007005044216888606AE0042061681B
:10229000A0FB015003461920A9FB007001462A4605
:1022A0003846FDF7ECFF824604206168A0FB015030
:1022B00003461920A9FB007001462A463846FDF75F
:1022C000DEFF6421B0FBF1F000EBC00101EB001078
:1022D000AAEB8000322101EB00106421B0FBF1F089
:1022E00000F0F00A04206168A0FB01700346192089
:1022F000A9FB00513A462846FDF7C1FF6421B0FB17
:10230000F1F00AEB001A04206168A0FB01510B46B2
:102310001920A9FB00712A463846FDF7B0FF834615
:1023200004206168A0FB015003461920A9FB00703E
:1023300001462A463846FDF7A2FF6421B0FBF1F0C2
:1023400000EBC00101EB0010ABEB8000322101EB90
:1023500000106421B0FBF1F000F00F005044216840
:102360008860BDE8F88F00000010014000140140B3
:1023700010B5034699629A85DA85002018642220F8
:1023800083F83E0000BF002083F83C0000BF1868BF
:10239000C06840F480701C68E0601868406940F0D4
:1023A00001001C6860611868C06840F020001C686B
:1023B000E060002010BD014691F83D00212828D1A1
:1023C0008868B0F5805F0BD1086948B90A6A10883F
:1023D000C0F308000B685860086A801C086205E0BA
:1023E0000B6A581C086218780B685860C88C401E2D
:1023F00080B2C88458B90868C06820F080000B68B3
:10240000D8600868C06840F040000B68D8600020C1
:1024100070470220FCE7000070B500240F4D104803
:10242000FFF71CFB00BF03E0641CAC4200D904E0D2
:102430000B48FFF709FB2028F6D100BF002403E07A
:10244000641CAC4200D906E0012206490448FFF7AB
:10245000CBFC0028F4D100BF70BD0000FFFF0100DD
:10246000E40000200E00002000BFFEE702480068E4
:10247000C0F30220704700000CED00E010B500280A
:1024800004DB0A07130E054A135406E00A07140E6C
:10249000034A00F00F031B1FD45410BD00E400E0FA
:1024A00018ED00E000BF70472DE9FF4107460C46DC
:1024B00015461E4600940195029669463846FEF779
:1024C0008DFABDE8FF81000010B504460723012204
:1024D00021460748FFF7E8FF0548FEF725FC0A21DB
:1024E0000348FEF7B9FB0248FEF73EFB80B210BD81
:1024F000280100202DE9F04107460C460025002662
:1025000008E03846FFF7E0FF0544052000F012F828
:10251000701CC6B2A642F4DBB5FBF4F0BDE8F08156
:1025200010B504460420FFF75FFA0148046010BDAF
:102530000400002070B504464FF4077094FBF0F5DA
:1025400094FBF0F100FB114603E0074800F00EF8A1
:102550006D1E002DF9D12EB14FF47A7106FB01F0FA
:1025600000F004F870BD0000603D080070B503463F
:1025700000224FF0E02675690D4E366803FB06F425
:102580004FF0E026B16910E04FF0E026B0698842D4
:102590000BD0884202D20E1A324402E02E1A0E44A8
:1025A00032440146A24200D300E0EDE700BF70BD17
:1025B0000400002000BF054A126802F04002002A11
:1025C000F9D0C2B2014B5A607047000000100140C0
:1025D00008B5FEF7D9FD0723022208214FF4A870A1
:1025E00000F03CF8FFF76AFCFEF7C2F8A820FFF7FE
:1025F00097FF4FF4E13000F09FF80BA0FDF7B6FE17
:1026000011E0FFF789FC00909DF800100BA0FDF78A
:10261000ADFE9DF801100DA0FDF7A8FE4FF47A70F5
:10262000FFF788FF00BFECE70D0AC4FAB7A2CBCDD5
:10263000B5C4CFFBCFA2CEAA3A0D0A00526573757E
:102640006C7420313A20307825780A005265737511
:102650006C7420323A20307825780A002DE9F04158
:1026600092B080460C4615461E460027302106A82B
:10267000FDF7E8FE142101A8FDF7E4FE00BF0020ED
:1026800000902A48006840F08050284908600846B9
:10269000006800F08050009000BF00BF00BF002025
:1026A00000902348006840F48040214908600846B3
:1026B000006800F48040009000BF00BF0120069039
:1026C0000004079002200C9041050D91CDF83C804C
:1026D0000E941095119606A8FEF738FF07461FB115
:1026E000012012B0BDE8F0810F200190022002907D
:1026F000002003904FF4A05004904FF480500590B8
:10270000052101A8FEF7E2FD07460FB10120E8E729
:10271000FEF722FD41F20101884205D1054800681B
:1027200040F48070034908600020DAE74038024036
:1027300000700040003C024010B5044609480A49B8
:1027400008600846446000218160C16001618161C8
:102750000C214161FFF7AAFA012204490248FFF760
:1027600043FB10BD00100140E40000200E000020DB
:10277000491058BFC1F140415B1058BFC3F14043FD
:102780008B42EFF30080704710F0004248BF404298
:10279000B0FA80F310FA03F10AD0C3F11D0303F578
:1027A00080634FEA415002EB035202EBD1217047A4
:1027B0004FF000007047000051EA030C17D41CF5DD
:1027C000801F58BFBCF5801F00F10680994218BFDA
:1027D000704708BF9042704707D711F5801F58BF58
:1027E00013F5801F19D499427047894270471CF530
:1027F000801F08D5BCF5801FF7D58B4218BF7047E6
:1028000008BF824270474FF4001C1CEB410F38BFD9
:102810001CEB430F01D28B42704770B500F0B2F849
:10282000922449004FF000514FF08053FFF7A0BFB2
:10283000DFF848C170B51CEA111E1EBF1CEA131553
:102840009EEA0C0F95EA0C0F00F06F8081EA0304FA
:1028500023EA4C134EEAD47E21EA4C1141F4801154
:1028600043F48013AE44A1FB024CA0FB0365AEF120
:102870007F7E361955EB0C05A1FB034C4CF1000390
:10288000A0FB021C16EB0C06654153F10003094244
:1028900018BF46F0010613F4007F0BD14FEA033155
:1028A0004FEA0530340341EA155140EA16506FF003
:1028B00003020AE04FEAC3214FEAC520F40241EACD
:1028C000555140EA56506FF0020202EB2E4201EBE6
:1028D000025585EACE710AD05FEA440C18BF24F095
:1028E000004450F1000041F1000120EAD47040F2B0
:1028F000FE7C624500D270BDA84214BF4FF08044F8
:102900004FF04044002E08BF0024BEF1806FA8BFE6
:10291000A1F1C041BDE8704080F282804FF000001C
:1029200001F1C04101F0004170479EEA0C0F0CEA32
:10293000131518BF95EA0C0F06D04FF0000081EA7E
:10294000030E0EF0004170BD00F01CF88900013E3E
:1029500000F007B800F009B84FEA430C5FEA5C5C8E
:1029600008D081EA030100F05BB84FEA410C5FEA4E
:102970005C5CF6D14FF00000014970470000FF0792
:102980000000F87F0EF1020E2EF0030E5EF8046BCD
:10299000364205D4012A43EB030515F5001F12D872
:1029A000012841EB010C1CF5001F0CD80ED14FEA99
:1029B000D17C15F5001F0CEB4C0C0CF1020C08BF80
:1029C0004CEBD37C04E04FF0080C01E04FEAD37CE1
:1029D0000CEB4C0526FA05F606F00706B6F1040CDA
:1029E00006D20EEB860CBDE870404CF0010C60473F
:1029F000DFE80CF0090B02024FF000414FF000003D
:102A0000A1F5002170BD19461046012851EB0104C3
:102A100018BFD4F5001484BF002001F0004170BD40
:102A20000808A0F500114FEA3101704753EA010C84
:102A300017D41CF5801F58BFBCF5801F00F106801D
:102A40008B4218BF704708BF8242704707D713F503
:102A5000801F58BF11F5801F19D48B4270479B42CD
:102A600070471CF5801F08D5BCF5801FF7D599422B
:102A700018BF704708BF904270474FF4001C1CEB12
:102A8000430F38BF1CEB410F01D2994270470FB47E
:102A90000CBC03BCFFF7C1BE4FF04070E1EE100A62
:102AA0007047000000000000000001020304060758
:102AB00008090000000001020304303132333435CC
:102AC000363738394142434445464030580030316A
:102AD0003233343536373839616263646566403085
:102AE00078000000042B0008000000201C000000FB
:102AF000C4010008202B00081C000020B4050000C1
:102B0000E00100080024F4000000000000000000C4
:102B100000000000000000001000000001000000A4
:040000050800018965
:00000001FF
